:020000040000FA
:42000000FFFF62F73300FFFFFFFFFFFFFFFFFFFFFFFFFFFFFFFFFFFFFFFFFFFFFFFFFFFFFFFFFFFFFFFFFFFFFFFFFFFFFFFFFFFFFFFFFFFFFFFFFFFFFFFFFFFFFFFFFFFFFFFF70
:42004200800C9001324006C80019001360024C8009324106C8001920034C80613001000000000006980013001324830C900132400618061360022002648001300006C00050FC85
:420084000015A00254800A50012A800A50012A4005B4800A50012A4005A8002DA00200000000000950012A800E780117E0025C800BD0022A400550012A400248000920013CFE56
:4200C6000004800010000240000800024000080001300002400008000100000000000000000000000000000000000000000000000000000000000000000000000000000010FC48
:42010800000000000000000000000000000000000000000000000000000000000000000000000000000000000000000000000000000000000000000000000000000000003CFE7B
:42014A000001200005A0001480020008000160000485A0001000025000000000000000000000000000000000080800000000000000000000000000000000000000000000D4FC43
:42018C00000580041000024000080802410008108120000250000A0000000000000000000000000000000000000000000000000000000000000000000000000000000000E8FE08
:4201CE00000000000000000240000000000000000000100000400000000000000000000000000000000000000000000000000000000000000000000000000000000000005CFD04
:42021000000000000000000000000000000000000000002000000300000000000000000000000000000000000000000000000000000000000000000000000000000000002CFD60
:42025200000000000000001EC0030000000000000000700000C080000000000000000000000000000000000000000000000000000000000000000000000000000000000034FFA6
:4202940000000000000000824490000000000000000090280040080000000000000000000000000000000000000000000000000000000000000000000000000000000000B8FC1E
:4202D600000000000000000000200000000000000000000800000800000000000000000000000000000000000000000000000000000000000000000000000000000000003CFC7E
:420318000000000000000006D0800000000000000000302000C0800000000000000000000000000000000000000000000000000000000000000000000000000000000000E0FEDF
:42035A000000000000000018040300000000000000004000000000000000000000000000000000000000000000000000000000000000000000000000000000000000000014FEF0
:42039C0000000000000000000040000000000000000040100040A00000000000000000000000000000000000000000000000000000000000000000000000000000000000C8FEE9
:4203DE00A0010401000000024100000000000000000010000040030000000000000000000000000000000000000000000000000000000000000000000000000000000000A0FC05
:4204200000000008000000000400000000000000000000000000000000000000000000000000000000000000000000000000000000000000000000000000000000000000F8FE98
:42046200E0011C080000000E00000000000000000000000000C0800000000000000000000000000000000000000000000000000000000000000000000000000000000000DCFE2B
:4204A400284004000000009204A000000000000000000000004008000000000000000000000000000000000000000000000000000000000000000000000000000000008000FCB0
:4204E600005030020000000000000000000000000000004200000800000000000000000000000000000000000000000000000000000000000000000000000000000000809CFFED
:42052800E0013C0800000006D0000200000000000000300000C0800000000000000000000000000000000000000000000000000000000000000000000000000000000000C8FC60
:42056A00040030080000000804000000000000000000C00000000000000000000000000000000000000000000000000000000000000000000000000000000000000000005DFCEE
:4205AC000044940000000008008B0000000000000000C0220040A000000000000000000000000000000000000000000000000000000000000000000000000000000000003CFDA7
:4205EE00200080000000000A450000000000000000001000004003000000000000000000000000000000000000000000000000000000000000000000000000000000000028FD64
:42063000000000100000000000000000000000000000000000000000000000000000000000000000000000000000000000000000000000000000000000000000000000003CFF3D
:42067200E0013C000000000EC0030000000000000000F00000C00000000000000000000000000000000000000000000000000000000000000000000000000000000000000CFF9D
:4206B400A4013400000000424488000000000000000010220040A300000000000000000000000000000000000000000000000000000000000000000000000000000000007DFD8E
:4206F6008C51B00000000000020000000000000000000042000020040000000000000000000000000000000000000000000000000000000000000000000000000000000008FCC9
:42073800E0013C0800000016C0000200000000000000300000C000000000000000000000000000000000000000000000000000000000000000000000000000000000000048FD4D
:42077A00080000080000000800030000000000000000C000000003000000000000000000000000000000000000000000000000000000000000000000000000000000008070FD72
:4207BC00004400010000000005400000000000000000001000008B0000000000000000000000000000000000000000000000000000000000000000000000000000000000C0FC1A
:4207FE00A00834000000000240100000000000000000100400400300000000000000000000000000000000000000000000000000000000000000000000000000000000009CFE9A
:4208400000410000000000000080000000000000000000200000030000000000000000000000000000000000000000000000000000000000000000000000000000000000F4FCA2
:4208820060403C000000001EC4010000000000000000700000C000000000000000000000000000000000000000000000000000000000000000000000000000000000000028FE1F
:4208C4002804040A00000002408A00000000000000009022004000000000000000000000000000000000000000000000000000000000000000000000000000000000008014FD69
:420906008048000A000000000200000000000000000000420000200400000000000000000000000000000000000000000000000000000000000000000000000000000080D0FE27
:42094800E0003C000000001EC0000200000000000000300000C0000000000000000000000000000000000000000000000000000000000000000000000000000000000000D0FCB5
:42098A0004403008000000000001000000000000000040000000030000000000000000000000000000000000000000000000000000000000000000000000000000000000F9FF73
:4209CC0000088400000000000541000000000000000040100000A30000000000000000000000000000000000000000000000000000000000000000000000000000000000ACFC7C
:420A0E00A00104000000000240000000000000000000D004004000000000000000000000000000000000000000000000000000000000000000000000000000000000000048FE65
:420A500080010000000000000080000000000000000080400000000000000000000000000000000000000000000000000000000000000000000000000000000000000000E4FFC0
:420A9200E00130000000000000000200000000000000C02000C0000000000000000000000000000000000000000000000000000000000000000000000000000000000000D0FCA3
:420AD400A40130000000004004100000000000000000C0020040000000000000000000000000000000000000000000000000000000000000000000000000000000000080F0FD48
:420B16000C4830020000000002200000000000000000C0020000230000000000000000000000000000000000000000000000000000000000000000000000000000000080D0FCC4
:420B580060003C0800000006C0800000000000000000F02000C083000000000000000000000000000000000000000000000000000000000000000000000000000000000034FDED
:420B9A00080000000000000000800000000000000000C0000000030000000000000000000000000000000000000000000000000000000000000000000000000000000000D9FCF9
:420BDC000000800800000018050A0000000000000000C0280040030000000000000000000000000000000000000000000000000000000000000000000000000000000000D8FC29
:420C1E00A0010400000000024000000000A00100000010000040890000000000000000000000000000000000000000000000000000000000000000000000000000000000B8FE7D
:420C60000000000000000000008000000080010000000000000002000000000000000000000000000000000000000000000000000000000000000000000000000000000014FD3E
:420CA20060403C000000001EC483000000E001000000F02000C0020000000000000000000000000000000000000000000000000000000000000000000000000000000000E8FD37
:420CE400A8053400000000024008000000A00100000010020040A200000000000000000000000000000000000000000000000000000000000000000000000000000000803CFC56
:420D26000040300A0000008004200000000044000000000800002104000000000000000000000000000000000000000000000000000000000000000000000000000000809CFEE2
:420D680060003C000000001EC0800000006000000000304000C0020000000000000000000000000000000000000000000000000000000000000000000000000000000000F0FCD1
:420DAA00044000080000000004010000000000000000C000000001000000000000000000000000000000000000000000000000000000000000000000000000000000000025FED2
:420DEC00001084000000004000410000000000000000001000008A0000000000000000000000000000000000000000000000000000000000000000000000000000000000CCFC4E
:420E2E00200034000000001A41030000002000000000D0000040000000000000000000000000000000000000000000000000000000000000000000000000000000000000ECFDB7
:420E700000003000000000180400000000000000000080200000000000000000000000000000000000000000000000000000000000000000000000000000000000000000F8FD5F
:420EB20000003C00000000180003000000E001000000C04000C000000000000000000000000000000000000000000000000000000000000000000000000000000000000048FCC2
:420EF4000450340000000098048B0000002020000000C0040040000000000000000000000000000000000000000000000000000000000000000000000000000000000080B8FF92
:420F36000C48000A0000008804030000000044000000C0080000030000000000000000000000000000000000000000000000000000000000000000000000000000000080D4FD2C
:420F780060000C000000001EC003010000E001000000F08000C083000000000000000000000000000000000000000000000000000000000000000000000000000000000074FEE3
:420FBA00084000000000001810030000000040000000C02000000300000000000000000000000000000000000000000000000000000000000000000000000000000000000DFD55
:420FFC00800504000000001801A30000000000000000C0080040030000000000000000000000000000000000000000000000000000000000000000000000000000000000F4FF70
:42103E002000B00000000002400000000020000000001000004000000000000000000000000000000000000000000000000000000000000000000000000000000000000044FCAE
:42108000000030100000000000000000000000000000002000000000000000000000000000000000000000000000000000000000000000000000000000000000000000002CFCA6
:4210C20000003C0000000000000000000000000000000000000080000000000000000000000000000000000000000000000000000000000000000000000000000000000040FDF3
:421104000840340000000000009000000000000000000028000008000000000000000000000000000000000000000000000000000000000000000000000000000000000031FD3F
:42114600005000080000008004200000000044000000004200000B000000000000000000000000000000000000000000000000000000000000000000000000000000000030FDAD
:4211880060000C0000000006C0800000006000000000300000C080000000000000000000000000000000000000000000000000000000000000000000000000000000000038FD6E
:4211CA00840100000000001804800000008041000000000000000000000000000000000000000000000000000000000000000000000000000000000000000000000000803CFE47
:42120C000044000000000058000B000000800100000080220000A0000000000000000000000000000000000000000000000000000000000000000000000000000000000038FD01
:42124E00000000000000000000000000000000000000000000000200000000000000000000000000000000000000000000000000000000000000000000000000000000001CFC44
:421290002000008000100002400008000120000480001000020000080001200004000000000010000240000800012000048000100002400008000120000480001000020034FCFE
:4212D200000020000000000000000000000000000000000000000000000000000000000000000000000000000000000000000000000000000000000000000000000000001CFCA2
:4213140024000480001000024000080001200004800010000240000800012000040000000000100002400008000120000480001000024000080001200004800010000280FCFCE9
:421356000C000000000000100002000000000100000080000000020000000000000000000000000000000000000000000000000000000000000000000000000000000080ECFD4B
:421398000000008000100000000008000100000480000000020000080001200004000000000010000240000800012000048000100002400008000120000480001000020030FD8A
:4213DA00080120000000000000000000000000000000000000000000000000000000000000000000000000000000000000000000000000000000000000000000000000009DFC0F
:42141C002000048000100002400008000120000480001000024000080001200004000000000010000240000800012000048000100002400008000120000480001000020034FC2C
:42145E00000000000000000000000000000000000000000000000000000000000000000000000000000000000000000000000000000000000000000000000000000000003CFE12
:4214A000000000000000000000000000000000000000000000000000000000000000000000000000000000000000000000000000000000000000000000000000000000003CFED0
:4214E200000000000000000000000000000000000000000000000000000000000000000000000000000000000000000000000000000000000000000000000000000000003CFE8E
:42152400000000000000000000000000000000000000000000000000000000000000000000000000000000000000000000000000000000000000000000000000000000003CFE4B
:42156600000000000000000000000000000000000000000000000000000000000000000000000000000000000000000000000000000000000000000000000000000000003CFE09
:4215A800000000000000000000000000000000000000000000000000000000000000000000000000000000000000000000000000000000000000000000000000000000003CFEC7
:4215EA00000000000000000000000000000000000000000000000000000000000000000000000000000000000000000000000000000000000000000000000000000000003CFE85
:42162C00000000000000000000000000000000000000000000000000000000000000000000000000000000000000000000000000000000000000000000000000000000003CFE42
:42166E00000000000000000000000000000000000000000000000000000000000000000000000000000000000000000000000000000000000000000000000000000000003CFE00
:4216B000000000000000000000000000000000000000000000000000000000000000000000000000000000000000000000000000000000000000000000000000000000003CFEBE
:4216F200000000000000000000000000000000000000000000000000000000000000000000000000000000000000000000000000000000000000000000000000000000003CFE7C
:42173400000000000000000000000000000000000000000000000000000000000000000000000000000000000000000000000000000000000000000000000000000000003CFE39
:421776000000000000000000040000000000000000000000000000000000000000000000000000000000000000000000000000000000000000000000000000000000000078FEB7
:4217B800000000000000000000000000000000000000000000000000000000000000000000000000000000000000000000000000000000000000000000000000000000003CFEB5
:4217FA0000000000000000000800000000000000000000000000000000000000000000000000000000000000000000000000000000000000000000000000000000000000B4FEF3
:42183C0000000000000000800000000000000000000000000000000000000000000000000000000000000000000000000000000000000000000000000000000000000000BCFE30
:42187E00000000000000000000000000000000000000000000000000000000000000000000000000000000000000000000000000000000000000000000000000000000003CFEEE
:4218C000000000000000000000000000000000000000000000000000000000000000000000000000000000000000000000000000000000000000000000000000000000003CFEAC
:42190200000000000000000000000000000000000000000000000000000000000000000000000000000000000000000000000000000000000000000000000000000000003CFE69
:42194400000000000000000000000000000000000000000000000000000000000000000000000000000000000000000000000000000000000000000000000000000000003CFE27
:42198600000000000000000000000000000000000000200000000000000000000000000000000000000000000000000000000000000000000000000000000000000000003CFCC7
:4219C800000000000000000000000000000000000000000000000000000000000000000000000000000000000000000000000000000000000000000000000000000000003CFEA3
:421A0A00000000000000000000000000000000000000000000000000000000000000000000000000000000000000000000000000000000000000000000000000000000003CFE60
:421A4C00000000000000000000000000000000000000000000000000000000000000000000000000000000000000000000000000000000000000000000000000000000003CFE1E
:421A8E00000000000000000000000000000000000000000000000000000000000000000000000000000000000000000000000000000000000000000000000000000000003CFEDC
:421AD000000000000000000000000000000000000000000000000000000000000000000000000000000000000000000000000000000000000000000000000000000000003CFE9A
:421B120000000000000000000008000000000000000000000000000000000000000000000000000000000000000000000000000000000000000000000000000000000000BCFECF
:421B540000000000000000000A00000000000000000000000000000000000000000000000000000000000000000000000000000000000000000000000000000000000000B4FC95
:421B9600000000000000000000000000000000000000000000000000000000000000000000000000000000000000000000000000000000000000000000000000000000003CFED3
:421BD800000000000000000000000000000000000000000000000000000000000000000000000000000000000000000000000000000000000000000000000000000000003CFE91
:421C1A00000000000000000000000000000000000000000000000000000000000000000000000000000000000000000000000000000000000000000000000000000000003CFE4E
:421C5C00000000000000000000000000000000000000000000000000000000000000000000000000000000000000000000000000000000000000000000000000000000003CFE0C
:421C9E0000000000000000000000000000000000000080010000000000000000000000000000000000000000000000000000000000000000000000000000000000000000A4FFE0
:421CE000000020000000000000000000000000000000000000000000000000000000000000000000000000000000000000000000000000000000000000000000000000001CFC8A
:421D2200000000000000000000000000000000000000000000000000000000000000000000000000000000000000000000000000000000000000000000000000000000003CFE45
:421D6400000000000000000000000000000000000000000000000000000000000000000000000000000000000000000000000000000000000000000000000000000000003CFE03
:421DA60000000000000000080081000000000000000040000000000000000000000000000000000000000000000000000000000000000000000000000000000000000000E8FE4C
:421DE800000000000000000000000000000000000000000000000000000000000000000000000000000000000000000000000000000000000000000000000000000000003CFE7F
:421E2A000043000600000004800001000000000000002000000401000000000000000000000000000000000000000000000000000000000000000000000000000000000060FF24
:421E6C00800800000000000804810000008000000000402080800000000000000000000000000000000000000000000000000000000000000000000000000000000000000CFE35
:421EAE008000000000000008048100000080000000004020000000000000000000000000000000000000000000000000000000000000000000000000000000000000000084FE83
:421EF000000000000000000000000000000000000000000000000000000000000000000000000000000000000000000000000000000000000000000000000000000000003CFE76
:421F3200000000000000000000000000000000000000000000000000000000000000000000000000000000000000000000000000000000000000000000000000000000003CFE33
:421F7400000000000000000000000000000000000000000000000000000000000000000000000000000000000000000000000000000000000000000000000000000000003CFEF1
:421FB6000000000000000000000000000000000000004040000000000000000000000000000000000000000000000000000000000000000000000000000000000000000038FE33
:421FF800000000000000000000000100000000000000000000000000000000000000000000000000000000000000000000000000000000000000000000000000000000002CFF7B
:42203A000A0000000000000000000000000000000000000000000000000000000000000000000000000000000000000000000000000000000000000000000000000000009CFEC0
:42207C00000000000000000000000000000000000000000000000000000000000000000000000000000000000000000000000000000000000000000000000000000000003CFEE8
:4220BE00000000000000000000000000000000000000000000000000000000000000000000000000000000000000000000000000000000000000000000000000000000003CFEA6
:42210000000000000000000000000000000000000000000000000000000000000000000000000000000000000000000000000000000000000000000000000000000000003CFE63
:422142000000000000000000400000000020000000001000000000000000000000000000000000000000000000000000000000000000000000000000000000000000000018FFD4
:42218400000000000000000200040000000000000000000000000002000000000000000000000000000000000000000000000000000000000000000000000000000000005CFEB7
:4221C600000000000000000000000000000000000000000000000000000000000000000000000000000000000000000000000000000000000000000000000000000000003CFE9D
:42220800000000000000000000000000000000000000000000000000000000000000000000000000000000000000000000000000000000000000000000000000000000003CFE5A
:42224A00000000000000000000000000000000000000000000000000000000000000000000000000000000000000000000000000000000000000000000000000000000003CFE18
:42228C00000000000000000000000000000000000000000000000000000000000000000000000000000000000000000000000000000000000000000000000000000000003CFED6
:4222CE00000000000000000000000000000000000000000000000000000000000000000000000000000000000000000000000000000000000000000000000000000000003CFE94
:42231000000000000000000000000000000000000000000000000000000000000000000000000000000000000000000000000000000000000000000000000000000000003CFE51
:42235200000000000000000000000000000000000000000000000000000000000000000000000000000000000000000000000000000000000000000000000000000000003CFE0F
:42239400000000000000000000000000000000000000000000000000000000000000000000000000000000000000000000000000000000000000000000000000000000003CFECD
:4223D600000000000000000000000000000000000000000000000000000000000000000000000000000000000000000000000000000000000000000000000000000000003CFE8B
:42241800000000000000000000000000000000000000000000000000000000000000000000000000000000000000000000000000000000000000000000000000000000003CFE48
:42245A00000000000000000000000000000000000000000000000000000000000000000000000000000000000000000000000000000000000000000000000000000000003CFE06
:42249C00000000000000000000000000000000000000000000000000000000000000000000000000000000000000000000000000000000000000000000000000000000003CFEC4
:4224DE00000000000000000000000000000000000000000000000000000000000000000000000000000000000000000000000000000000000000000000000000000000003CFE82
:422520000800000000000000000000000000000000000000000000000000000000000000000000000000000000000000000000000000000000000000000000000000008034FEBF
:4225620000000000000000000000000000000000000000000000000000000000000000000000000000000000000000000000000000000000000000000000000000000080B4FE05
:4225A400000000000000000000000000000000000000000000000000000000000000000000000000000000000000000000000000000000000000000000000000000000003CFEBB
:4225E600040000000000000000000000000000000000000000000000000000000000000000000000000000000000000000000000000000000000000000000000000000006DFF43
:42262800000000000000000000000000000000000000000000000000000000000000000000000000000000000000000000000000000000000000000000000000000000003CFE36
:42266A00000000000000000000000000000000000000000000000000000000000000000000000000000000000000000000000000000000000000000000000000000000003CFEF4
:4226AC00000000000000000000000000000000000000000000000000000000000000000000000000000000000000000000000000000000000000000000000000000000003CFEB2
:4226EE00000000000000000000000000000000000000000000000000000000000000000000000000000000000000000000000000000000000000000000000000000000003CFE70
:42273000040000000000000000000000000000000000000000000000000000000000000000000000000000000000000000000000000000000000000000000000000000006DFFF7
:422772000C000000000000000000000000000000000000000000000000000000000000000000000000000000000000000000000000000000000000000000000000000000FCFE1F
:4227B400000000000000000000000000000000000000000000000000000000000000000000000000000000000000000000000000000000000000000000000000000000003CFEA9
:4227F6000800000000000000000000000000000000000000000000000000000000000000000000000000000000000000000000000000000000000000000000000000008034FEE7
:42283800000000000000000000000000000000000000000000000000000000000000000000000000000000000000000000000000000000000000000000000000000000003CFE24
:42287A00000000000000000000000000000000000000000000000000000000000000000000000000000000000000000000000000000000000000000000000000000000003CFEE2
:4228BC00000000000000000000000000000000000000000000000000000000000000000000000000000000000000000000000000000000000000000000000000000000003CFEA0
:4228FE00000000000000000000000000000000000000000000000000000000000000000000000000000000000000000000000000000000000000000000000000000000003CFE5E
:42294000040000000000000000000000000000000000000000000000000000000000000000000000000000000000000000000000000000000000000000000000000000006DFFE5
:422982000C000000000000000000000000000000000000000000000000000000000000000000000000000000000000000000000000000000000000000000000000000000FCFE0D
:4229C400000000000000000000000000000000000000000000000000000000000000000000000000000000000000000000000000000000000000000000000000000000003CFE97
:422A06000800000000000000000000000000000000000000000000000000000000000000000000000000000000000000000000000000000000000000000000000000008034FED4
:422A4800000000000000000000000000000000000000000000000000000000000000000000000000000000000000000000000000000000000000000000000000000000003CFE12
:422A8A00000000000000000000000000000000000000000000000000000000000000000000000000000000000000000000000000000000000000000000000000000000003CFED0
:422ACC00000000000000000000000000000000000000000000000000000000000000000000000000000000000000000000000000000000000000000000000000000000003CFE8E
:422B0E00000000000000000000000000000000000000000000000000000000000000000000000000000000000000000000000000000000000000000000000000000000003CFE4B
:422B500004000000000000000000000000000000000000000000000000000000000000000000000000000000000000000000000000000000000000000000000000000080F4FECD
:422B92000C00000000000000000000000000000000000000000000000000000000000000000000000000000000000000000000000000000000000000000000000000008074FE03
:422BD400000000000000000000000000000000000000000000000000000000000000000000000000000000000000000000000000000000000000000000000000000000003CFE85
:422C160008000000000000000000000000000000000000000000000000000000000000000000000000000000000000000000000000000000000000000000000000000000ADFFC8
:422C5800000000000000000000000000000000000000000000000000000000000000000000000000000000000000000000000000000000000000000000000000000000003CFE00
:422C9A00000000000000000000000000000000000000000000000000000000000000000000000000000000000000000000000000000000000000000000000000000000003CFEBE
:422CDC00000000000000000000000000000000000000000000000000000000000000000000000000000000000000000000000000000000000000000000000000000000003CFE7C
:422D1E00000000000000000000000000000000000000000000000000000000000000000000000000000000000000000000000000000000000000000000000000000000003CFE39
:422D6000040000000000000000000000000000000000000000000000000000000000000000000000000000000000000000000000000000000000000000000000000000006DFFC1
:422DA2000C000000000000000000000000000000000000000000000000000000000000000000000000000000000000000000000000000000000000000000000000000000FCFEE9
:422DE400000000000000000000000000000000000000000000000000000000000000000000000000000000000000000000000000000000000000000000000000000000003CFE73
:422E26000800000000000000000000000000000000000000000000000000000000000000000000000000000000000000000000000000000000000000000000000000008034FEB0
:422E6800000000000000000000000000000000000000000000000000000000000000000000000000000000000000000000000000000000000000000000000000000000003CFEEE
:422EAA00000000000000000000000000000000000000000000000000000000000000000000000000000000000000000000000000000000000000000000000000000000003CFEAC
:422EEC00000000000000000000000000000000000000000000000000000000000000000000000000000000000000000000000000000000000000000000000000000000003CFE6A
:422F2E00000000000000000000000000000000000000000000000000000000000000000000000000000000000000000000000000000000000000000000000000000000003CFE27
:422F700004000000000000000000000000000000000000000000000000000000000000000000000000000000000000000000000000000000000000000000000000000080E5FFB7
:422FB2000C00000000000000000000000000000000000000000000000000000000000000000000000000000000000000000000000000000000000000000000000000008074FEDF
:422FF400000000000000000000000000000000000000000000000000000000000000000000000000000000000000000000000000000000000000000000000000000000003CFE61
:423036000800000000000000000000000000000000000000000000000000000000000000000000000000000000000000000000000000000000000000000000000000008025FFAC
:42307800000000000000000000000000000000000000000000000000000000000000000000000000000000000000000000000000000000000000000000000000000000003CFEDC
:4230BA00000000000000000000000000000000000000000000000000000000000000000000000000000000000000000000000000000000000000000000000000000000003CFE9A
:4230FC00000000000000000000000000000000000000000000000000000000000000000000000000000000000000000000000000000000000000000000000000000000003CFE58
:42313E00000000000000000000000000000000000000000000000000000000000000000000000000000000000000000000000000000000000000000000000000000000003CFE15
:4231800008000000000000000000000000000000000000000000000000000000000000000000000000000000000000000000000000000000000000000000000000000000ADFF59
:4231C200000000000000000000000000000000000000000000000000000000000000000000000000000000000000000000000000000000000000000000000000000000003CFE91
:42320400000000000000000000000000000000000000000000000000000000000000000000000000000000000000000000000000000000000000000000000000000000003CFE4E
:4232460004000000000000000000000000000000000000000000000000000000000000000000000000000000000000000000000000000000000000000000000000000080F4FED0
:42328800000000000000000000000000000000000000000000000000000000000000000000000000000000000000000000000000000000000000000000000000000000003CFECA
:4232CA00000000000000000000000000000000000000000000000000000000000000000000000000000000000000000000000000000000000000000000000000000000003CFE88
:42330C002000048000100002400008000120000480001000024000080001200004000000000010000240000800012000048000100002400008000120000480001000020034FC1D
:42334E00000000000000000000000000000000000000000000000000000000000000000000000000000000000000000000000000000000000000000000000000000000003CFE03
:4233900024000480001000024000080001200004800010000240000800012000040000000000100002400008000120000480001000024000080001200004800010000280EDFD5B
:4233D2000C00000000000000000000000000000000000000000000000000000000000000000000000000000000000000000000000000000000000000000000000000008074FEBB
:423414002000048000100002400008000120000480001000024000080001200004000000000010000240000800012000048000100002400008000120000480001000020034FC14
:423456000800000000000000000000000000000000000000000000000000000000000000000000000000000000000000000000000000000000000000000000000000008025FF88
:423498002000048000100002400008000120000480001000024000080001200004000000000010000240000800012000048000100002400008000120000480001000020034FC90
:4234DA00000000000000000000000000000000000000000000000000000000000000000000000000000000000000000000000000000000000000000000000000000000003CFE76
:42351C00000000000000000000000000000000000000000000000000000000000000000000000000000000000000000000000000000000000000000000000000000000003CFE33
:42355E00000000000000000000000000000000000000000000000000000000000000000000000000000000000000000000000000000000000000000000000000000000003CFEF1
:4235A000000000000000000000000000000000000000000000000000000000000000000000000000000000000000000000000000000000000000000000000000000000003CFEAF
:4235E200000000000000000000000000000000000000000000000000000000000000000000000000000000000000000000000000000000000000000000000000000000003CFE6D
:42362400000000000000000000000000000000000000000000000000000000000000000000000000000000000000000000000000000000000000000000000000000000003CFE2A
:42366600000000000000000000000000000000000000000000000000000000000000000000000000000000000000000000000000000000000000000000000000000000003CFEE8
:4236A800000000000000000000000000000000000000000000000000000000000000000000000000000000000000000000000000000000000000000000000000000000003CFEA6
:4236EA00000000000000000000000000000000000000000000000000000000000000000000000000000000000000000000000000000000000000000000000000000000003CFE64
:42372C00000000000000000000000000000000000000000000000000000000000000000000000000000000000000000000000000000000000000000000000000000000003CFE21
:42376E00000000000000000000000000000000000000000000000000000000000000000000000000000000000000000000000000000000000000000000000000000000003CFEDF
:4237B000000000000000000000000000000000000000000000000000000000000000000000000000000000000000000000000000000000000000000000000000000000003CFE9D
:4237F200000000000000000000000000000000000000000000000000000000000000000000000000000000000000000000000000000000000000000000000000000000003CFE5B
:42383400000000000000000000000000000000000000000000000000000000000000000000000000000000000000000000000000000000000000000000000000000000003CFE18
:42387600000000000000000000000000000000000000000000000000000000000000000000000000000000000000000000000000000000000000000000000000000000003CFED6
:4238B800000000000000000000000000000000000000000000000000000000000000000000000000000000000000000000000000000000000000000000000000000000003CFE94
:4238FA00000000000000000000000000000000000000000000000000000000000000000000000000000000000000000000000000000000000000000000000000000000003CFE52
:42393C00000000000000000000000000000000000000000000000000000000000000000000000000000000000000000000000000000000000000000000000000000000003CFE0F
:42397E00000000000000000000000000000000000000000000000000000000000000000000000000000000000000000000000000000000000000000000000000000000003CFECD
:4239C000000000000000000000000000000000000000000000000000000000000000000000000000000000000000000000000000000000000000000000000000000000003CFE8B
:423A0200000000000000000000000000000000000000000000000000000000000000000000000000000000000000000000000000000000000000000000000000000000003CFE48
:423A4400000000000000000000000000000000000000000000000000000000000000000000000000000000000000000000000000000000000000000000000000000000003CFE06
:423A8600000000000000000000000000000000000000000000000000000000000000000000000000000000000000000000000000000000000000000000000000000000003CFEC4
:423AC800000000000000000000000000000000000000000000000000000000000000000000000000000000000000000000000000000000000000000000000000000000003CFE82
:423B0A00000000000000000000000000000000000000000000000000000000000000000000000000000000000000000000000000000000000000000000000000000000003CFE3F
:423B4C00000000000000000000000000000000000000000000000000000000000000000000000000000000000000000000000000000000000000000000000000000000003CFEFD
:423B8E00000000000000000000000000000000000000000000000000000000000000000000000000000000000000000000000000000000000000000000000000000000003CFEBB
:423BD000000000000000000000000000000000000000000000000000000000000000000000000000000000000000000000000000000000000000000000000000000000003CFE79
:423C1200000000000000000000000000000000000000000000000000000000000000000000000000000000000000000000000000000000000000000000000000000000003CFE36
:423C5400000000000000000000000000000000000000000000000000000000000000000000000000000000000000000000000000000000000000000000000000000000003CFEF4
:423C9600000000000000000000000000000000000000000000000000000000000000000000000000000000000000000000000000000000000000000000000000000000003CFEB2
:423CD800000000000000000000000000000000000000000000000000000000000000000000000000000000000000000000000000000000000000000000000000000000003CFE70
:423D1A00000000000000000000000000000000000000000000000000000000000000000000000000000000000000000000000000000000000000000000000000000000003CFE2D
:423D5C00000000000000000000000000000000000000000000000000000000000000000000000000000000000000000000000000000000000000000000000000000000003CFEEB
:423D9E00000000000000000000000000000000000000000000000000000000000000000000000000000000000000000000000000000000000000000000000000000000003CFEA9
:423DE000000000000000000000000000000000000000000000000000000000000000000000000000000000000000000000000000000000000000000000000000000000003CFE67
:423E2200000000000000000000000000000000000000000000000000000000000000000000000000000000000000000000000000000000000000000000000000000000003CFE24
:423E6400000000000000000000000000000000000000000000000000000000000000000000000000000000000000000000000000000000000000000000000000000000003CFEE2
:423EA600000000000000000000000000000000000000000000000000000000000000000000000000000000000000000000000000000000000000000000000000000000003CFEA0
:423EE800000000000000000000000000000000000000000000000000000000000000000000000000000000000000000000000000000000000000000000000000000000003CFE5E
:423F2A00000000000000000000000000000000000000000000000000000000000000000000000000000000000000000000000000000000000000000000000000000000003CFE1B
:423F6C00000000000000000000000000000000000000000000000000000000000000000000000000000000000000000000000000000000000000000000000000000000003CFED9
:423FAE00000000000000000000000000000000000000000000000000000000000000000000000000000000000000000000000000000000000000000000000000000000003CFE97
:423FF000000000000000000000000000000000000000000000000000000000000000000000000000000000000000000000000000000000000000000000000000000000003CFE55
:42403200000000000000000000000000000000000000000000000000000000000000000000000000000000000000000000000000000000000000000000000000000000003CFE12
:42407400000000000000000000000000000000000000000000000000000000000000000000000000000000000000000000000000000000000000000000000000000000003CFED0
:4240B600000000000000000000000000000000000000000000000000000000000000000000000000000000000000000000000000000000000000000000000000000000003CFE8E
:4240F800000000000000000000000000000000000000000000000000000000000000000000000000000000000000000000000000000000000000000000000000000000003CFE4C
:42413A00000000000000000000000000000000000000000000000000000000000000000000000000000000000000000000000000000000000000000000000000000000003CFE09
:42417C00000000000000000000000000000000000000000000000000000000000000000000000000000000000000000000000000000000000000000000000000000000003CFEC7
:4241BE00000000000000000000000000000000000000000000000000000000000000000000000000000000000000000000000000000000000000000000000000000000003CFE85
:42420000000000000000000000000000000000000000000000000000000000000000000000000000000000000000000000000000000000000000000000000000000000003CFE42
:42424200000000000000000000000000000000000000000000000000000000000000000000000000000000000000000000000000000000000000000000000000000000003CFE00
:42428400000000000000000000000000000000000000000000000000000000000000000000000000000000000000000000000000000000000000000000000000000000003CFEBE
:4242C600000000000000000000000000000000000000000000000000000000000000000000000000000000000000000000000000000000000000000000000000000000003CFE7C
:42430800000000000000000000000000000000000000000000000000000000000000000000000000000000000000000000000000000000000000000000000000000000003CFE39
:42434A00000000000000000000000000000000000000000000000000000000000000000000000000000000000000000000000000000000000000000000000000000000003CFEF7
:42438C00000000000000000000000000000000000000000000000000000000000000000000000000000000000000000000000000000000000000000000000000000000003CFEB5
:4243CE00000000000000000000000000000000000000000000000000000000000000000000000000000000000000000000000000000000000000000000000000000000003CFE73
:42441000000000000000000000000000000000000000000000000000000000000000000000000000000000000000000000000000000000000000000000000000000000003CFE30
:42445200000000000000000000000000000000000000000000000000000000000000000000000000000000000000000000000000000000000000000000000000000000003CFEEE
:42449400000000000000000000000000000000000000000000000000000000000000000000000000000000000000000000000000000000000000000000000000000000003CFEAC
:4244D600000000000000000000000000000000000000000000000000000000000000000000000000000000000000000000000000000000000000000000000000000000003CFE6A
:42451800000000000000000000000000000000000000000000000000000000000000000000000000000000000000000000000000000000000000000000000000000000003CFE27
:42455A00000000000000000000000000000000000000000000000000000000000000000000000000000000000000000000000000000000000000000000000000000000003CFEE5
:42459C000800000000000000000000000000000000000000000000000000000000000000000000000000000000000000000000000000000000000000000000000000008034FE23
:4245DE0000000000000000000000000000000000000000000000000000000000000000000000000000000000000000000000000000000000000000000000000000000080B4FE69
:42462000000000000000000000000000000000000000000000000000000000000000000000000000000000000000000000000000000000000000000000000000000000003CFE1E
:42466200040000000000000000000000000000000000000000000000000000000000000000000000000000000000000000000000000000000000000000000000000000006DFFA6
:4246A400000000000000000000000000000000000000000000000000000000000000000000000000000000000000000000000000000000000000000000000000000000003CFE9A
:4246E600000000000000000000000000000000000000000000000000000000000000000000000000000000000000000000000000000000000000000000000000000000003CFE58
:42472800000000000000000000000000000000000000000000000000000000000000000000000000000000000000000000000000000000000000000000000000000000003CFE15
:42476A00000000000000000000000000000000000000000000000000000000000000000000000000000000000000000000000000000000000000000000000000000000003CFED3
:4247AC00040000000000000000000000000000000000000000000000000000000000000000000000000000000000000000000000000000000000000000000000000000006DFF5B
:4247EE000C000000000000000000000000000000000000000000000000000000000000000000000000000000000000000000000000000000000000000000000000000000FCFE83
:42483000000000000000000000000000000000000000000000000000000000000000000000000000000000000000000000000000000000000000000000000000000000003CFE0C
:424872000800000000000000000000000000000000000000000000000000000000000000000000000000000000000000000000000000000000000000000000000000008034FE4A
:4248B400000000000000000000000000000000000000000000000000000000000000000000000000000000000000000000000000000000000000000000000000000000003CFE88
:4248F600000000000000000000000000000000000000000000000000000000000000000000000000000000000000000000000000000000000000000000000000000000003CFE46
:42493800000000000000000000000000000000000000000000000000000000000000000000000000000000000000000000000000000000000000000000000000000000003CFE03
:42497A00000000000000000000000000000000000000000000000000000000000000000000000000000000000000000000000000000000000000000000000000000000003CFEC1
:4249BC00040000000000000000000000000000000000000000000000000000000000000000000000000000000000000000000000000000000000000000000000000000006DFF49
:4249FE000C000000000000000000000000000000000000000000000000000000000000000000000000000000000000000000000000000000000000000000000000000000FCFE71
:424A4000000000000000000000000000000000000000000000000000000000000000000000000000000000000000000000000000000000000000000000000000000000003CFEFA
:424A82000800000000000000000000000000000000000000000000000000000000000000000000000000000000000000000000000000000000000000000000000000008034FE38
:424AC400000000000000000000000000000000000000000000000000000000000000000000000000000000000000000000000000000000000000000000000000000000003CFE76
:424B0600000000000000000000000000000000000000000000000000000000000000000000000000000000000000000000000000000000000000000000000000000000003CFE33
:424B4800000000000000000000000000000000000000000000000000000000000000000000000000000000000000000000000000000000000000000000000000000000003CFEF1
:424B8A00000000000000000000000000000000000000000000000000000000000000000000000000000000000000000000000000000000000000000000000000000000003CFEAF
:424BCC0004000000000000000000000000000000000000000000000000000000000000000000000000000000000000000000000000000000000000000000000000000080F4FE31
:424C0E000C00000000000000000000000000000000000000000000000000000000000000000000000000000000000000000000000000000000000000000000000000008074FE66
:424C5000000000000000000000000000000000000000000000000000000000000000000000000000000000000000000000000000000000000000000000000000000000003CFEE8
:424C920008000000000000000000000000000000000000000000000000000000000000000000000000000000000000000000000000000000000000000000000000000000ADFF2C
:424CD400000000000000000000000000000000000000000000000000000000000000000000000000000000000000000000000000000000000000000000000000000000003CFE64
:424D1600000000000000000000000000000000000000000000000000000000000000000000000000000000000000000000000000000000000000000000000000000000003CFE21
:424D5800000000000000000000000000000000000000000000000000000000000000000000000000000000000000000000000000000000000000000000000000000000003CFEDF
:424D9A00000000000000000000000000000000000000000000000000000000000000000000000000000000000000000000000000000000000000000000000000000000003CFE9D
:424DDC00040000000000000000000000000000000000000000000000000000000000000000000000000000000000000000000000000000000000000000000000000000006DFF25
:424E1E000C000000000000000000000000000000000000000000000000000000000000000000000000000000000000000000000000000000000000000000000000000000FCFE4C
:424E6000000000000000000000000000000000000000000000000000000000000000000000000000000000000000000000000000000000000000000000000000000000003CFED6
:424EA2000800000000000000000000000000000000000000000000000000000000000000000000000000000000000000000000000000000000000000000000000000008034FE14
:424EE400000000000000000000000000000000000000000000000000000000000000000000000000000000000000000000000000000000000000000000000000000000003CFE52
:424F2600000000000000000000000000000000000000000000000000000000000000000000000000000000000000000000000000000000000000000000000000000000003CFE0F
:424F6800000000000000000000000000000000000000000000000000000000000000000000000000000000000000000000000000000000000000000000000000000000003CFECD
:424FAA00000000000000000000000000000000000000000000000000000000000000000000000000000000000000000000000000000000000000000000000000000000003CFE8B
:424FEC0004000000000000000000000000000000000000000000000000000000000000000000000000000000000000000000000000000000000000000000000000000080F4FE0D
:42502E000C00000000000000000000000000000000000000000000000000000000000000000000000000000000000000000000000000000000000000000000000000008074FE42
:42507000000000000000000000000000000000000000000000000000000000000000000000000000000000000000000000000000000000000000000000000000000000003CFEC4
:4250B20008000000000000000000000000000000000000000000000000000000000000000000000000000000000000000000000000000000000000000000000000000000ADFF08
:4250F400000000000000000000000000000000000000000000000000000000000000000000000000000000000000000000000000000000000000000000000000000000003CFE40
:42513600000000000000000000000000000000000000000000000000000000000000000000000000000000000000000000000000000000000000000000000000000000003CFEFD
:42517800000000000000000000000000000000000000000000000000000000000000000000000000000000000000000000000000000000000000000000000000000000003CFEBB
:4251BA00000000000000000000000000000000000000000000000000000000000000000000000000000000000000000000000000000000000000000000000000000000003CFE79
:4251FC00040000000000000000000000000000000000000000000000000000000000000000000000000000000000000000000000000000000000000000000000000000006DFF01
:42523E000C000000000000000000000000000000000000000000000000000000000000000000000000000000000000000000000000000000000000000000000000000000FCFE28
:42528000000000000000000000000000000000000000000000000000000000000000000000000000000000000000000000000000000000000000000000000000000000003CFEB2
:4252C2000800000000000000000000000000000000000000000000000000000000000000000000000000000000000000000000000000000000000000000000000000008034FEF0
:42530400000000000000000000000000000000000000000000000000000000000000000000000000000000000000000000000000000000000000000000000000000000003CFE2D
:42534600000000000000000000000000000000000000000000000000000000000000000000000000000000000000000000000000000000000000000000000000000000003CFEEB
:425388002000048000100002400008000120000480001000024000080001200004000000000010000240000800012000048000100002400008000120000480001000020034FC81
:4253CA00000000000000000000000000000000000000000000000000000000000000000000000000000000000000000000000000000000000000000000000000000000003CFE67
:42540C0024000480001000024000080001200004800010000240000800012000040000000000100002400008000120000480001000024000080001200004800010000280FCFCB0
:42544E000C00000000000000000000000000000000000000000000000000000000000000000000000000000000000000000000000000000000000000000000000000008074FE1E
:425490002000048000100002400008000120000480001000024000080001200004000000000010000240000800012000048000100002400008000120000480001000020034FC78
:4254D20008000000000000000000000000000000000000000000000000000000000000000000000000000000000000000000000000000000000000000000000000000000ADFFE4
:425514002000048000100002400008000120000480001000024000080001200004000000000010000240000800012000048000100002400008000120000480001000020034FCF3
:42555600000000000000000000000000000000000000000000000000000000000000000000000000000000000000000000000000000000000000000000000000000000003CFED9
:42559800000000000000000000000000000000000000000000000000000000000000000000000000000000000000000000000000000000000000000000000000000000003CFE97
:4255DA00000000000000000000000000000000000000000000000000000000000000000000000000000000000000000000000000000000000000000000000000000000003CFE55
:42561C00000000000000000000000000000000000000000000000000000000000000000000000000000000000000000000000000000000000000000000000000000000003CFE12
:42565E00000000000000000000000000000000000000000000000000000000000000000000000000000000000000000000000000000000000000000000000000000000003CFED0
:4256A000000000000000000000000000000000000000000000000000000000000000000000000000000000000000000000000000000000000000000000000000000000003CFE8E
:4256E200000000000000000000000000000000000000000000000000000000000000000000000000000000000000000000000000000000000000000000000000000000003CFE4C
:42572400000000000000000000000000000000000000000000000000000000000000000000000000000000000000000000000000000000000000000000000000000000003CFE09
:42576600000000000000000000000000000000000000000000000000000000000000000000000000000000000000000000000000000000000000000000000000000000003CFEC7
:4257A800000000000000000000000000000000000000000000000000000000000000000000000000000000000000000000000000000000000000000000000000000000003CFE85
:4257EA00000000000000000000000000000000000000000000000000000000000000000000000000000000000000000000000000000000000000000000000000000000003CFE43
:42582C00000000000000000000000000000000000000000000000000000000000000000000000000000000000000000000000000000000000000000000000000000000003CFE00
:42586E00000000000000000000000000000000000000000000000000000000000000000000000000000000000000000000000000000000000000000000000000000000003CFEBE
:4258B000000000000000000000000000000000000000000000000000000000000000000000000000000000000000000000000000000000000000000000000000000000003CFE7C
:4258F200000000000000000000000000000000000000000000000000000000000000000000000000000000000000000000000000000000000000000000000000000000003CFE3A
:42593400000000000000000000000000000000000000000000000000000000000000000000000000000000000000000000000000000000000000000000000000000000003CFEF7
:42597600000000000000000000000000000000000000000000000000000000000000000000000000000000000000000000000000000000000000000000000000000000003CFEB5
:4259B800000000000000000000000000000000000000000000000000000000000000000000000000000000000000000000000000000000000000000000000000000000003CFE73
:4259FA00000000000000000000000000000000000000000000000000000000000000000000000000000000000000000000000000000000000000000000000000000000003CFE31
:425A3C00000000000000000000000000000000000000000000000000000000000000000000000000000000000000000000000000000000000000000000000000000000003CFEEE
:425A7E00000000000000000000000000000000000000000000000000000000000000000000000000000000000000000000000000000000000000000000000000000000003CFEAC
:425AC000000000000000000000000000000000000000000000000000000000000000000000000000000000000000000000000000000000000000000000000000000000003CFE6A
:425B0200000000000000000000000000000000000000000000000000000000000000000000000000000000000000000000000000000000000000000000000000000000003CFE27
:425B4400000000000000000000000000000000000000000000000000000000000000000000000000000000000000000000000000000000000000000000000000000000003CFEE5
:425B8600000000000000000000000000000000000000000000000000000000000000000000000000000000000000000000000000000000000000000000000000000000003CFEA3
:425BC800000000000000000000000000000000000000000000000000000000000000000000000000000000000000000000000000000000000000000000000000000000003CFE61
:425C0A00000000000000000000000000000000000000000000000000000000000000000000000000000000000000000000000000000000000000000000000000000000003CFE1E
:425C4C00000000000000000000000000000000000000000000000000000000000000000000000000000000000000000000000000000000000000000000000000000000003CFEDC
:425C8E00000000000000000000000000000000000000000000000000000000000000000000000000000000000000000000000000000000000000000000000000000000003CFE9A
:425CD000000000000000000000000000000000000000000000000000000000000000000000000000000000000000000000000000000000000000000000000000000000003CFE58
:425D1200000000000000000000000000000000000000000000000000000000000000000000000000000000000000000000000000000000000000000000000000000000003CFE15
:425D5400000000000000000000000000000000000000000000000000000000000000000000000000000000000000000000000000000000000000000000000000000000003CFED3
:425D9600000000000000000000000000000000000000000000000000000000000000000000000000000000000000000000000000000000000000000000000000000000003CFE91
:425DD800000000000000000000000000000000000000000000000000000000000000000000000000000000000000000000000000000000000000000000000000000000003CFE4F
:425E1A00000000000000000000000000000000000000000000000000000000000000000000000000000000000000000000000000000000000000000000000000000000003CFE0C
:425E5C00000000000000000000000000000000000000000000000000000000000000000000000000000000000000000000000000000000000000000000000000000000003CFECA
:425E9E00000000000000000000000000000000000000000000000000000000000000000000000000000000000000000000000000000000000000000000000000000000003CFE88
:425EE000000000000000000000000000000000000000000000000000000000000000000000000000000000000000000000000000000000000000000000000000000000003CFE46
:425F2200000000000000000000000000000000000000000000000000000000000000000000000000000000000000000000000000000000000000000000000000000000003CFE03
:425F6400000000000000000000000000000000000000000000000000000000000000000000000000000000000000000000000000000000000000000000000000000000003CFEC1
:425FA600000000000000000000000000000000000000000000000000000000000000000000000000000000000000000000000000000000000000000000000000000000003CFE7F
:425FE800000000000000000000000000000000000000000000000000000000000000000000000000000000000000000000000000000000000000000000000000000000003CFE3D
:42602A00000000000000000000000000000000000000000000000000000000000000000000000000000000000000000000000000000000000000000000000000000000003CFEFA
:42606C00000000000000000000000000000000000000000000000000000000000000000000000000000000000000000000000000000000000000000000000000000000003CFEB8
:4260AE00000000000000000000000000000000000000000000000000000000000000000000000000000000000000000000000000000000000000000000000000000000003CFE76
:4260F000000000000000000000000000000000000000000000000000000000000000000000000000000000000000000000000000000000000000000000000000000000003CFE34
:42613200000000000000000000000000000000000000000000000000000000000000000000000000000000000000000000000000000000000000000000000000000000003CFEF1
:42617400000000000000000000000000000000000000000000000000000000000000000000000000000000000000000000000000000000000000000000000000000000003CFEAF
:4261B600000000000000000000000000000000000000000000000000000000000000000000000000000000000000000000000000000000000000000000000000000000003CFE6D
:4261F800000000000000000000000000000000000000000000000000000000000000000000000000000000000000000000000000000000000000000000000000000000003CFE2B
:42623A00000000000000000000000000000000000000000000000000000000000000000000000000000000000000000000000000000000000000000000000000000000003CFEE8
:42627C00000000000000000000000000000000000000000000000000000000000000000000000000000000000000000000000000000000000000000000000000000000003CFEA6
:4262BE00000000000000000000000000000000000000000000000000000000000000000000000000000000000000000000000000000000000000000000000000000000003CFE64
:42630000000000000000000000000000000000000000000000000000000000000000000000000000000000000000000000000000000000000000000000000000000000003CFE21
:426342000000040000100002000000000120000080001000024000000045A008000000000000000002400100000100040480000000000000000001000404000000000000FCFD55
:426384000000000000000000000000000000000000000000000000000008048100000000000000000000820000000080000000000000000000000000800000000000000068FC64
:4263C6000000001000004000080000000004800000000240000800010007E480000000000000000006C00100000360000C8001000000000000000360000C000000000000E8FEF7
:426408000000300100C00498000000004C8009000026C00498001300000DA001000000000000000002408200000120000480000000000000000001200004000000000000A8FC7B
:42644A0000000002000008000100000020000800004000020001200000848144000000000000000058001100008C8411300246000000000000008C80093002000000000044FFA5
:42648C0000003C0800F0201E040000000FE441008007F1201EC48300000FE00100000000000000001E848200000FE0413C8807010000000000000FE2413C080000000000CCFCD9
:4264CE000000300000C00018080000000C8001000006C40018080301000C8001000000000000000018000100000C8001300006000000000000000C800130000000000000A4FF38
:426510000000301100C01018010000000C8245000006C02018002300004C824900000000000000001A008900000C8001300006000000000000000C800130000000000000B8FF3A
:426552002000048000000240000008000021000000100010400008000045000414020000000010000240030001012000048000000000000000000100040400005008000050FF86
:4265940000000000000040000800000000000000000002000008000100080480200800000000000000000000200000000000000000000000000000008000000080200000BCFFC3
:4265D60000800C000032000600000020038001008001300006C00000000764001C0000000000300006C00318000360000C8001000000000000000360000C00007000000060FEDF
:42661800880904002610000200006002010010018000100002400000000D2000A4080000000010000240800800012000048000000000000000000120000400009028008094FFE5
:42665A000004302210C00458100000024C82010000C6C08018110B0100048045100000000000C00498001060014C8005B00016000000000000004C8005B000004048008078FE24
:42669C00E0413C8007F1401E000078100F6040008007F0001EC00300000FE201282000000000F0201E848378100FE8413C8807010000000000000FE2413C0800A000000074FD78
:4266DE008401300006C00018000060000C8041000006C00018000300000C8001100000000000C00018000360000C8001300006000000000000000C80013000004020000095FC90
:4267200080893400A6C00018000060110D8011000006C00018000300000CA201100A00000000C00018008860000C8001300006000000000000000C800130000040080000BCFD82
:426762000004040010100002000000080D00200480000002024000000045A00834000000000010004040000800202000040010000000000808000120000400000010000040FC40
:4267A4000080000000020000000000000000000000000040000000000008048100000000000000000008000000000400000000020000000001000000000000000000000070FFE6
:4267E6006000009001004000080018000F60000010003200000800010007E4803C0000000000300006C00318000360000C8001000000C00018000360000C00003000000078FED1
:426828002400308100C0049800000800212200300126100098001300000DA001840800000000100002400308000120000480000000004000080001200004000010000000A5FD45
:42686A008C050209C600224004006000208805020110C1084004880000448048000000000000C00498001360124C8009300116010000001360024C8009300100C0240000ACFC5E
:4268AC00E0013C8007F0001E000078200EE0013C8807F0801EC00300000FE201382000000000F0201E848378000FE8413C9007000000C08378100FE2413C1000F00000009CFD81
:4268EE008801300006C00018000060000C8201300006C00018000300000C8001300000000000002018000060000C800130000600000000036000008201300000C000008030FF34
:426930008001300A06C0281805006000808001301146C1001805A300002C8245000A00000000000218008860000C800130000600000000036000808001300000D000000044FC90
:426972002000008400100002400000010100048080001000024000680045A0080400000000001000024000000120200004001000000040000001012000040000D000000020FD42
:4269B40000000000000000000000002000008000100000000000000000080281000000000000000000000000200004000000000200000000002000000000000000000000D4FE4E
:4269F60000800C0000320006000019000064000C8001004006C00078000FE2803C0000000000300006000018000360000C8001000000C00018000360000C0000F000000010FDE4
:426A38008809040026100002001308004C2000048000C00402400008148DA00134000000000010000200000800012000048000000000400008000120000400001028008074FD6B
:426A7A000040B00840C124980490600400808530122601209804930004848400300000000000C02218030862128C8009310046010000009360424C824930000000480080E0FC0E
:426ABC00E0013C8007F0001EC00378200FE4013C8007F0001EC003704007E041382000000000F0001EC00078000FE2013C8807000000C00378000FE0013C0800E0000000A8FEDB
:426AFE008441300006C10018000361000C8001300006C02018000360100C8001000000000000C00018008360000C8001300006000000000360000C8001300000C020000035FCB4
:426B40008011340046C00018000360000C8801300006C00818000300048C8451000A00000000C00018002360000C8001300006000000000360000C800130000000080000A0FFCB
:426B82002000808000100002000808000120000480001000024000080045A0080004000000001000404000080020000480001010000040000800012000800000100000008CFDC1
:426BC4000000001000000000000001000000000000000000000000000008048100000000000000000008000000000480001000020000000000000000000010000000000020FD26
:426C060060000C8001300006C00000200F0080009001300006C000780007E4800C0000000000300006C00318000360000C8001300000C00018000360000C0000F0000000E8FEF6
:426C48002800048000100002400060020D8009308100100002400068000DA0010400000000001000024003080001200004800010000040000800012000040000D0000080B0FC7C
:426C8A008045302116C11018032300142C0840000216C4225810236204848008B00000000000C00818030B62000C8005300006C12200008B60112C8231B01000C048008014FF2A
:426CCC00E0013C8007F0001EC00379000EE0013C9007F0001EC00370400FE2413C0800000000F0201E800378400FE2413C8807F00000C00378000FE0013C0000E00000006CFFD7
:426D0E008401300006C0001800036010008241300806C00018000300100C8241300000000000C00018008060000C8001300006C00000000360000C80013000000020000029FCB2
:426D50008001340006C0001800036001808005B00006C00018000300048C8011340000000000C00018002060000C8001300006C00000000360000C800130000000080000C4FF59
:426D92003000048000100002400008002522000480001000024000000845A00800040000000010004000400800202000808000100000400000010100048080000010020008FC57
:426DD4000000300000000000000000000800000000000000000000000008048100000000000000000008000000000400001000000000000000200000800010000000000028FEC6
:426E160060003C8801300006000019000760000C8001300006C000180007E4800C0000000000300006C00018000360000C8001300000C00018000360000C80013000060068FCBD
:426E5800240084800010000200130800292200048000100002400008000DA00104000000000010000240000800012000048000100000400008000120000480001000028054FFE7
:426E9A008431000646C2201805806040248851300A06C1081805A36012248040300100000000C02818010B60018C8411300146C12800004360028C8449300246C104188540FD46
:426EDC00E001388007F0001EC00378000AE0013C8007F0401EC00378000FE2013C0800000000F0001EC48378100FE0413C9007F00000C00378200FE0013C8807F0201E002CFEE0
:426F1E008C01002006C0001800036000048201300006C00018000360000C8241300000000000C00018000360000C8001300006C00000000360000C8001300006C0001800D9FFB8
:426F60008001B00006C0001800536000848001300006C00018000368002C8005340000000000C00018400360000C8001300006C00000000360000C8001308006D0001A00B4FD8B
:426FA2002000348000100002400008000120000480001000024000000845A008000400000000100002004008000120008080001000024000080001200080001000104000C4FDF8
:426FE4000000000000000000000000000000000000000000000000000008048100000000000000000000000000000000001000000000000000000000000010000200000858FF5D
:427026008001008801C00006000318000C60000C0006C00006C000180007E4800C0000000000300006C00018000360000C8001300006C00018000360000C800130000600C8FCB4
:42706800041081800000880200200A00802800040040048802400008000DA00104000000000010000240000800012000048000100002400008000120000480001000028045FED6
:4270AA008C11000646C40018011360220C8001B10006C00018000B6402248204300200000000C04898042360028C8001B00006C14058081360120C8005B00006C00818830CFF59
:4270EC0060400C800730201EC880780003E2013CA00131201EC80378100FE0413C0800000000F0001EC08378100FE2413C8807F0001EC08378000FE2413C8807F4201E0044FEF8
:42712E008801002006C00018008360000C8001300006C00018000360000C8241300000000000C00018000360000C8001300006C00018000360000C8001300006C000188021FD46
:427170008051800006C02218000B60008C8201300016C12818000368000C8001340000000000C0001A400368000C8001300006C00018000360000C8001300006D0001800E0FC95
:4271B2002000048000100002400008002122000480001000024000080045A00804020000000010000200400800010004808000100002400008000120008080001008020014FC85
:4271F40000000000000000000000000000000000000000000000000000080481000800000000000000000000000000800010000000000000000000000000100000200000D0FF35
:427236006000300006300018C00060000060003080013000180003000007E480000000000000300006C00018000360000C8001300006C00018000360000C800100000600E0FF70
:4272780024000022401400005100004420220000A200100000112002140DA00180080000000010000240000800012000048000100002400008000120000480000028020009FE05
:4272BA008C05B00046C0421800136104208809B00046C0441800030004848210000000000000C00218010360042C8009300216C22418050B60012C80113000160148580464FFE0
:4272FC00E0010D8801F10006C403181003E0810C8807F20006C48018400FE0810C2000000000F0201EC48378100FE2413C8807F0001EC08378100FE2413C880730001E00F4FDB5
:42733E008801300006C0001800036010008201300806C00018000300100C8241000000000000C00018000360000C8001300006C00018000360000C80013000060020188088FD4F
:427380008001300946C1005804036004888001300206C00058048B60044C8009200A00000000C00018400368000D8001300006C00018400360000CA00130800680081A0040FDF8
:4273C200000000000000000000000000000000000000000000000000000000000000000000000000000000000000000000000000000000000000000000000000000000003CFE4F
:427404002000008000100002400008000020000480001000024000000001000000000000000010000000000000002000048000100002000008000100000400000000000088FCFE
:427446000000200000000000000000000800000000000000000000400000000120000000000000001000024000080000000000000000000200000000010000048000100098FFF3
:42748800280004800010000240000800012000048000100002400008000120000400000000001000024000080001200004800010000240000800012000048000100002802DFDDE
:4274CA0000010041048000100002400040100120000480001000020041000000802000000000800000001004000000012000040000100000400000000020000000820080C4FF92
:42750C00000000000000000000000000000000000000000000000000000000000000000000000000000000000000000000000000000000000000000000000000000000003CFE03
:42754E0004002000000000000000000008000000000000000000004000080001200000000000000010000240000800000000008000000002000008000100000480001080C1FEAE
:4275900020000080001000024000080000200004800010000240000000012000000000000000100002000008000120000480001000024000080001200004800000000200ACFD3F
:4275D200000000000000000000000000000000000000000000000000000000000000000000000000000000000000000000000000000000000000000000000000000000003CFE3D
:42761400000000000000000000000000000000000000000000000000000000000000000000000000000000000000000000000000000000000000000000000000000000003CFEFA
:427656000000060000000000000000000000000000000000000000000000000000000000000000000000000000000000000000000000000000000000000000000000000078FC78
:42769800000000040000000000000000000000000000000000000000000000000000000000000000000000000000000000000000000000000000000000000000000000007CFE32
:4276DA00000000000000000000000000000000000000000000000000000000000000000000000000000000000000000000000000000000000000000000000000000000003CFE34
:42771C00000000000000000000010000000000000000000000000000000000000000000000000000000000000000000000000000000000000000000000000000000000002CFE00
:42775E00000000000000000000000000000000000000000000000000000000000000000000000000000000000000000000000000000000000000000000000000000000003CFEAF
:4277A000000000000000000000000000000000000000000000000000000000000000000000000000000000000000000000000000000000000000000000000000000000003CFE6D
:4277E20000000004000000000000800000000000000000400000000000000000000000000000000000000000000000000000000000000000000000000000000000000000BCFEE7
:427824000000000000000000000000000000000000000000400000000000000000000000000000000000000000000000000000000000000000000000000000000000000038FEAC
:4278660000000000000000000000000000000000000800000000000000000000000000000000000000000000000000000000000000000000000000000000000000000000B4FE26
:4278A8000000000000000000000000000000004000000000000008000000000000000000000000000000000000000000000000000000000000000000000000000000000070FEE8
:4278EA000000000000000000000000000000000000000000040000010004024000000000000000000000000000000000000000000000000000000000000000000000000038FDDC
:42792C000000000000000000000020000000000000000000000000000000000000000000000000000004000000000000000000000000000000000000400000004000000058FE1F
:42796E0000000000000000000000080000000000000000000400000100020480000000000000000000100000000000000005000000000000000000000001000010000000CCFC56
:4279B00000000000000000000000000100008000000000000002000000048240001200000000000000000000000800001001040000000000000000000010000000000000C0FE4F
:4279F2000000000000000000000000000000000000000000000000000004824000000000000000000000000000000000100000000000000000000000001000000000000064FC0D
:427A340000000000000000000000000000000000000000000008000000000000000000000000000000000000000400000000020000000000000000000000000000000000D8FC2E
:427A760000000000000000000000000000000000000000000000000008000000000400000000000000000000000000000000000000000000000000000000000000100000E8FECC
:427AB80000000040000000000000800000100000000000000000000000000000000000000000000000000004000000000000000000000000000000000000000000000000A8FE12
:427AFA00000000000000000000000000008000000000000000000000000000000000000000000000000000000000000000000200000000000000000000100000000000009CFD1F
:427B3C000000000000000000000000000000000000000000000000000000000000000000000000000000000000000020000000000000000000080000000000000000000094FE4D
:427B7E00000000000000000000000000000000000000000000000000000000000000000000000000000000000000000000000000000000000000000000000000000000003CFE8B
:427BC000000000000000000000000000000000000000000000000000000000000000000000000000000000000000000000000000000000000000000000000000000000003CFE49
:427C02000000000000400000000000000000000000000000000000000000000000000000000000000000000000000000000000000000000000000000000000000000000038FECA
:427C440000000000000000000000000008000000000000000000000000000000000000000000000000000000000000000000000000000000000000000000000000000000BCFE3C
:427C8600000000000000000000000000000000000000000000000000200000000000000000000000000000000000000000000000000000000000000000000000000000003CFC64
:427CC800000000000000000000000000000000000000000000000000000000000000000000000000000000002000000000000000000000000000000000000000020000003CFE1E
:427D0A00000000000000000200000000000001000000000000000000000000000000000000000000000000000000000000000000000000000000000000000000000000001CFD1B
:427D4C00000000000000000040000000000000000000400000000000000000000000000000000000000000000000000000000000000000000000000000000000200000007CFCDD
:427D8E00000000000000000000000000000400400000000000000000000000000000000000000000000000000000000000000000000000000000000000000000000000007CFEF5
:427DD0000040800001000000000000001000000000000000000000000000000000000000000000000000000000000000000000000000000000000000000000000000000064FE3E
:427E12004000080001A00004800410000241000A000120000480000000000002000000000000000000000000000000002000000000000000000000200000000000000200A8FFD0
:427E54000000000000000000800000000000000000000000000000000000000000000000000000000000000000000001200004000000000040000000002000000000000040FFA8
:427E9600000000000000002000000000000000000000000000000000000000000000000000000000000000000000000000000000000000000000000000000000000000001CFE70
:427ED800000000000000000000002000000000000000000000000000000000000000000000000000000000000000000000000000000000000000000000000000000000001CFE2E
:427F1A004000101000000000000000000000000000000000000202200004024010080000000000200000000000040040000000000000000100000480000000000000000064FEF8
:427F5C000020000000000000000000000000000000000000000000000000000000000000000040000000812000008200100800010000000020000000001008004000000000FCD3
:427F9E004000091014800250000A20000400000000028002008800100002048008100000000010400040000A000228800420000400008000080002400004200010000004ACFF61
:427FE00020020022100002400008000128020008000000000240412010048250100600000000400208824040100801410804004000100002400004008120040440009000D4FF5B
:4280220000000000000000000000000000020000000000000000022010048240100000000000400008000000100000400000004000000000000004000000000040000000D4FF23
:4280640000000000000000000000000004000000000000000000000100000000000800000000000000048020000482000008000000080001200000800010080200000800ACFE26
:4280A600200000000000000000000001000000000000000000000000000000000000000000000000000000000000000000000000000000000000000000000000000000003CFD3E
:4280E80000004400100000000000080001200000080010000400010800000000040000000000000000400000000000000000000000000000000000000000000010000000C4FF9D
:42812A0000000080000000000200000000000000000000000000010000000000000000000000000000004000000000000000000000080000400000000020000000000000E8FF01
:42816C000001208004800018000240000000012000048000100002000002400100100000000000000000000000020000000000000000000000000000000000000000000028FC22
:4281AE0000000000000000000000000000000400800000000002000000010000000000000000000000000000000000000000000000000000000000000000000000000000C8FF41
:4281F000000000000000000000000000000000000000000000000000000000000000000000000000000000000000000000000000000000000000000000000000000000003CFE13
:428232000000000000000000000000000000000000800000000000000000000000000000000000000000000000000000000000000000000000000000000000000000000034FE58
:42827400000000000000000000000000000000000010000000000000000000000000000000000000000000000000000000000000000000000000000000000000000000002CFF8D
:4282B60000400008001120000480001000024000080001200004800000080001000000000000000002000000000002000000002000000000000000000000000000000000D4FD8C
:4282F8000002000000000000000000000000000800000000000000000000000000000000000000001000004000080000000000000000400200000000010000040000100020FD6E
:42833A000000000000000000000000000000000000000003000000040000000000000000000000000000000000000000000000000000000000000000000000000000000048FDB5
:42837C00000000000010000000000000000000000000000020000000000000000000000000002000000000000000000000000000000000000000020000000000000000000CFD64
:4283BE000000000000000000000000000000000080000000000000080000000000000000000000000000000000000000000000000000000000000000000000000000000034FEC3
:42840000000000000000000000000000000000000000000000000000000000000000000000000000000000000000000000000000000000000000000000000000000000003CFE00
:42844200000000000000000000000000000000000000020000000000200000000000000000000000000000000000000000000000000000000000000000000000000000001CFCBE
:42848400000000000000000000000000000000000026000000000060020000000000000000000000000000000000000000000000000000000000000000000000000000005CFCD6
:4284C6000000000000000000000000000000000000400000000000000400000000000000000000000000000000000000000000000000000000000000000000000000000078FEBA
:428508000000000000000000000000000000000080070100000000781000000000000000000000000000000000000000000000000000000000000000000000000000000054FFCE
:42854A00000000000000000000000000000000000006040000000060000000000000000000000000000000000000000000000000000000000000000000000000000000001CFE6B
:42858C0000000000000000000000000000000000004600000000006008000000000000000000000000000000000000000000000000000000000000000000000000000000D8FE29
:4285CE0000000000000000000000000000000000001000000000000801000000000000000000000000000000000000000000000000000000000000000000000000000000B4FF9F
:42861000000000000000000000000000000000000000020000000000100000000000000000000000000000000000000000000000000000000000000000000000000000001CFFFB
:428652000000000000000000000000000000000080010000000000380000000000000000000000000000000000000000000000000000000000000000000000000000000004FC2D
:42869400080000000000000000000000000000008000000000000008140000000000000000000000000000000000000000000000000000000000000000000000000000807CFF05
:4286D6000000000000000000000000000000000000060000000000600400000000000000000000000000000000000000000000000000000000000000000000000000008094FEE6
:428718000000000000000000000000000000000080070200000000781000000000000000000000000000000000000000000000000000000000000000000000000000000064FFAB
:42875A00040000000000000000000000000000000006000000000060100000000000000000000000000000000000000000000000000000000000000000000000000000000DFE58
:42879C000000000000000000000000000000000000060000000000200400000000000000000000000000000000000000000000000000000000000000000000000000000018FE5B
:4287DE000000000000000000000000000000000080000000000000680000000000000000000000000000000000000000000000000000000000000000000000000000000010FC65
:42882000000000000000000000000000000000000000000000000000000000000000000000000000000000000000000000000000000000000000000000000000000000003CFEDC
:4288620000000000000000000000000000000000000002000000007800000000000000000000000000000000000000000000000000000000000000000000000000000000A0FDBD
:4288A4000400000000000000000000000000000000260000000000081100000000000000000000000000000000000000000000000000000000000000000000000000000091FEC0
:4288E6000C000000000000000000000000000000001001000000000012000000000000000000000000000000000000000000000000000000000000000000000000000000DCFE47
:428928000000000000000000000000000000000080070000000000780000000000000000000000000000000000000000000000000000000000000000000000000000000044FECC
:42896A000800000000000000000000000000000000060000000000600000000000000000000000000000000000000000000000000000000000000000000000000000008054FE8B
:4289AC00000000000000000000000000000000000046010000000000140000000000000000000000000000000000000000000000000000000000000000000000000000002CFD05
:4289EE000000000000000000000000000000000080000000000000080000000000000000000000000000000000000000000000000000000000000000000000000000000034FE8D
:428A3000000000000000000000000000000000000000000000000000000000000000000000000000000000000000000000000000000000000000000000000000000000003CFECA
:428A72000000000000000000000000000000000080010000000000780000000000000000000000000000000000000000000000000000000000000000000000000000000000FCCD
:428AB4000800000000000000000000000000000080000000000000680000000000000000000000000000000000000000000000000000000000000000000000000000008018FCFC
:428AF60000000000000000000000000000000000002601000000006012000000000000000000000000000000000000000000000000000000000000000000000000000080C4FD64
:428B38000000000000000000000000000000000080070000000000780000000000000000000000000000000000000000000000000000000000000000000000000000000044FEBA
:428B7A000400000000000000000000000000000000060000000000000000000000000000000000000000000000000000000000000000000000000000000000000000000029FD89
:428BBC000000000000000000000000000000000000060000000000001400000000000000000000000000000000000000000000000000000000000000000000000000000038FD28
:428BFE00000000000000000000006800000000008000000000000008000000000000000000000000000000000000000000000000000000000000000000000000000000005CFEEB
:428C4000000000000000000000000000000000000000000000000000000000000000000000000000000000000000000000000000000000000000000000000000000000003CFEB8
:428C820000000000000000000000781000000000800100000000000010000000000000000000000000000000000000000000000000000000000000000000000000000000D4FFC4
:428CC4000400000000000000000008040000000080000000000000000100000000000000000000000000000000000000000000000000000000000000000000000000008028FE37
:428D06000C000000000000000000001100000000002608000000000041000000000000000000000000000000000000000000000000000000000000000000000000000080D4FE4D
:428D48000000000000000000000078000000000080070000000000180000000000000000000000000000000000000000000000000000000000000000000000000000000018FCBE
:428D8A000800000000000000000060100000000000060000000000001000000000000000000000000000000000000000000000000000000000000000000000000000000099FD83
:428DCC00000000000000000000000000000000000006000000000060020000000000000000000000000000000000000000000000000000000000000000000000000000007CFE83
:428E0E000000000000000000000068000000000080000000000000680000000000000000000000000000000000000000000000000000000000000000000000000000000078FC5E
:428E5000000000000000000000006000000000000000000000000000000000000000000000000000000000000000000000000000000000000000000000000000000000005CFE26
:428E92000000000000000000000078000000000080010000000000781000000000000000000000000000000000000000000000000000000000000000000000000000000078FDA8
:428ED4000800000000000000000068000000000080000000000000080100000000000000000000000000000000000000000000000000000000000000000000000000008044FEA1
:428F160000000000000000000000001100000000000601000000000041000000000000000000000000000000000000000000000000000000000000000000000000000080A4FCA0
:428F5800000000000000000000001800000000008007000000000078000000000000000000000000000000000000000000000000000000000000000000000000000000005CFE66
:428F9A00040000000000000000000000000000000006000000000060100000000000000000000000000000000000000000000000000000000000000000000000000000000DFE10
:428FDC000000000000000000000000000000000000060000000000000200000000000000000000000000000000000000000000000000000000000000000000000000000058FCF7
:42901E00000000000000000000000800000000008000000000000008020000000000000000000000000000000000000000000000000000000000000000000000000000001CFE64
:429060000000000000000000000000000000000000000000000000004000000000000000000000000000000000000000000000000000000000000000000000000000000078FE18
:4290A2000000000000000000000078000000000000060000000000002000000000000000000000000000000000000000000000000000000000000000000000000000000000FEF0
:4290E40004000000000000000000680000000000004004000000002002000000000000000000000000000000000000000000000000000000000000000000000000000080D8FC24
:429126000C00000000000000000060110000000000060000000000200000000000000000000000000000000000000000000000000000000000000000000000000000008060FE86
:429168000000000000000000000078000000000080010100000000581000000000000000000000000000000000000000000000000000000000000000000000000000000048FF1C
:4291AA0008000000000000000000001000000000000600000000006020000000000000000000000000000000000000000000000000000000000000000000000000000000DDFC0C
:4291EC00000000000000000000000000000000000016010000000040010000000000000000000000000000000000000000000000000000000000000000000000000000006CFD80
:42922E00000000000000000000000800000000008000000000000008000000000000000000000000000000000000000000000000000000000000000000000000000000003CFE34
:42927000000000000000000000000000000000000000000000000000000000000000000000000000000000000000000000000000000000000000000000000000000000003CFE82
:4292B2000000000000000000000000100000000080010000000000780000000000000000000000000000000000000000000000000000000000000000000000000000000010FD64
:4292F4000400000000000000000000040000000080000000000000680000000000000000000000000000000000000000000000000000000000000000000000000000000005FD46
:429336000C000000000000000000001100000000008600000000006041000000000000000000000000000000000000000000000000000000000000000000000000000000D0FEE3
:42937800000000000000000000001800000000008007000000000078000000000000000000000000000000000000000000000000000000000000000000000000000000005CFE42
:4293BA000800000000000000000000100000000000060000000000001000000000000000000000000000000000000000000000000000000000000000000000000000008060FC67
:4293FC000000000000000000000060000000000000060000000000000200000000000000000000000000000000000000000000000000000000000000000000000000000038FC93
:42943E00000000000000000000000000000000000000000000000000000000000000000000000000000000000000000000000000000000000000000000000000000000003CFEB2
:429480002000048000100002400008000120000480001000024000080001200004000000000010000240000800012000048000100002400008000120000480001000020034FC48
:4294C200000000000000000000000000000000000000000000000000000000000000000000000000000000000000000000000000000000000000000000000000000000003CFE2E
:42950400280004800010000240000800012000048000100002400008000120000400000000001000024000080001200004800010000240000800012000048000100002803CFC33
:4295460000000000000000000000400000000000000400000000004000000000000000000000000000000000000000000000000000000000000000000000000000000080B4FE2D
:429588002000048000100002400000000120000400001000024000000001200004000000000010000240000800012000048000100002400008000120000480001000020034FCCF
:4295CA00040000000000000000000000000000000000000000000000000000000000000000000000000000000000000000000000000000000000000000000000000000006DFFEF
:42960C002000048000100002400008000120000480001000024000080001200004000000000010000240000800012000048000100002400008000120000480001000020034FCBA
:42964E00000000000000000000000000000000000000000000000000000000000000000000000000000000000000000000000000000000000000000000000000000000003CFEA0
:42969000000000000000000000000000000000000000000000000000000000000000000000000000000000000000000000000000000000000000000000000000000000003CFE5E
:4296D200000000000000000000000000000000000000000000000000000000000000000000000000000000000000000000000000000000000000000000000000000000003CFE1C
:4297140000000000000000000000000000000000000800000000000000000000000000000000000000000000000000000000000000000000000000000000000000000000B4FE59
:42975600000000000000000000000000000000000000000000000000000000000000000000000000000000000000000000000000000000000000000000000000000000003CFE97
:42979800000000000000000000000000000000000000000000000000000000000000000000000000000000000000000000000000000000000000000000000000000000003CFE55
:4297DA00000000000000000000000000000000000000000000000000000000000000000000000000000000000000000000000000000000000000000000000000000000003CFE13
:42981C00000000000000000000000000000000000000000000000000000000000000000000000000000000000000000000000000000000000000000000000000000000003CFED0
:42985E00000000000000000000000000000000000000000000000000000000000000000000000000000000000000000000000000000000000000000000000000000000003CFE8E
:4298A000000000000000000000000000000000000000000000000000000000000000000000000000000000000000000000000000000000000000000000000000000000003CFE4C
:4298E200000000000000000000000000000000000000000000000000000000000000000000000000000000000000000000000000000000000000000000000000000000003CFE0A
:42992400000000000000000000000000000000000000000000000000000000000000000000000000000000000000000000000000000000000000000000000000000000003CFEC7
:42996600000000000000000000000000000000000000000000000000000000000000000000000000000000000000000000000000000000000000000000000000000000003CFE85
:4299A800000000000000000000000000000000000000000000000000000000000000000000000000000000000000000000100000000000000000000000000000000000003CFF32
:4299EA00000000000000000000000000000000000000000000000000000000000000000000000000000000000000000000200000000000000000000000000000000000003CFCE3
:429A2C0000000000000000000000000000000000000000000000000000000000000800000000000000000000000000000000000000000000000000000000000000000000B4FE3E
:429A6E000000000000000000000000000000000000000000000000000000000000040000000000000000000000000000000000000000000000000000000000000000000078FE3C
:429AB000000000000000000000000000000000000000000000000000000000000000000000000000000000000000000000000000000000000000000000000000000000003CFE3A
:429AF200000000000000000000000000000000000000000000000000000000000000000000000000000000000000000000000000000000000000000000000000000000003CFEF8
:429B3400000000000000000000000000000000000000000000000000000000000000000000000000000000000000000000000000000000000000000000000000000000003CFEB5
:429B7600000000000000000000000000000000000000000000000000000000000000000000000000000000000000000000000000000000000000000000000000000000003CFE73
:429BB800000000000000000000000000000000000000000000000000000000000000000000000000000000000000000000000000000000000000000000000000000000003CFE31
:429BFA00000000000000000000000000000000000000000000000000000000000000000000000000000000000000000000000000000000000000000000000000000000003CFEEF
:429C3C00000000000000000000000000000000000000000000000000000000000000000000000000000000000000000000000000000000000000000000000000000000003CFEAC
:429C7E0000000000000000000000000000000000000000000000000800000000000000000000000000000000000000000000000000000000000000000000000000000000B4FEEA
:429CC000000000000000000000000000000000000000000000000000000000000000000000000000000000000000000000000000000000000000000000000000000000003CFE28
:429D0200000000000000000000000000000000000000000000000000000000000000000000000000000000000000000000000000000000000000000000000000000000003CFEE5
:429D4400000000000000000000000000000000000000000000000000000000000000000000000000000000000000000000000000000000000000000000000000000000003CFEA3
:429D8600000000000000000000000000000000000000000000000000000000000000000000000000000000000000000000000000000000000000000000000000000000003CFE61
:429DC800000000000000000000000000000000000000000000000000000000000000000000000000000000000000000000000000000000000000000000000000000000003CFE1F
:429E0A00000000000000000000000000000000000000000000000020000000000000000000000000000000000000000000000000000000000000000000000000000000001CFCDE
:429E4C0000000000000000000000000000000000000008000000000000000000000000000000000000000000000000000000000000000000000000000000000000000000BCFE12
:429E8E00000000000000000000000000000000000001000000000010000000000000000000000000000000000000000000000000000000000000000000000000000000002CFE57
:429ED000000000000000000000000000000000000000000000000000000000000000000000000000000000000000000000000000000000000000000000000000000000003CFE16
:429F1200000000000000000000000000000000000000000000000000000000000000000000000000000000000000000000000000000000000000000000000000000000003CFED3
:429F54000000000000000000000000000000000000800000000000000000000000000000000000000000000000000000000000000000000000000000000000000000000034FE19
:429F96004000001000000000000000000000000000000000000000000000000000000000000000000000000000000000000000000000000000000000000000000000000078FFC2
:429FD800000000000000000000000000000000000000000000000000000000000000000000000000000000000000000000000000000000000000000000000000000000021CFE2B
:42A01A004000001000000000000000000000000000020000000000200000000000000000000000000000000000000000000000000000000000000000000000000000001058FE2C
:42A05C00000000000000000000002000000000000000000000000100000000000000000000000000000002000000000020000000000000000000000020000000000000000CFD56
:42A09E00000000000000000000002000000000000000000000000200000000000000000000000000000000000000000000000000000000000000000000000000000000003CFC26
:42A0E000000000000000000000000000000000000000000000000000000000000000000000000000000002000000000020000000000000000000000020000000000000003CFCC4
:42A12200100000000000000000000000000000000000000000000000000000000000000000000000000000000000000000000000000000000000000000000000000000001EFDD0
:42A1640000000000000000000000000000000000800000000000000000000000000000000000000000000000000000000000000000000000000000000000000000000000BCFE7F
:42A1A60000000000000000000000000000000000000000000000000008000000000000000000000000000000000000000000000000000000000000000000000000000000BCFEB5
:42A1E80004000000000000000000000000000000000400000000000000000000000000000000000000000000000000000000000000000000000000000000000000000080B0FEFF
:42A22A00040000000000000000000000000000000000000000000000000000000000000000000000000000000000000000000000000000000000000000000000000000007CFE74
:42A26C00000000000000000000000000000000000000000000000000000000000000000000000000000000000000000000000000000000000000000000000000000000003CFE76
:42A2AE00000000000000000000000000000000000000000000000000000000000000000000000000000000000000000000000000000000000000000000000000000000003CFE34
:42A2F000000000000000000000000000000000000000000000000000000000000000000000000000000000000000000000000000000000000000000000000000000000003CFEF2
:42A33200000000000000000000000000000000000000010000000000100000000000000000000000000000000000000000000000000000000000000000000000000000002CFFAD
:42A37400000000000000000000000000000000000000000000000000000000000000000000000000000000000000000000000000000000000000000000000000000000003CFE6D
:42A3B600000000000000000000000000000000000000000000000000000000000000000000000000000000000000000000000000000000000000000000000000000000003CFE2B
:42A3F800000000000000000000000000000000000000000000000000000000000000000000000000000000000000000000000000000000000000000000000000000000003CFEE9
:42A43A000000008000000000000000000000000000000000024003080000000000000000000000000000000000000000000000000000000000000000000000000000000048FFCC
:42A47C00000000000000000000000000000000000000000000040300000000000000000000000000000000000000000000000000000000000000000000000000000000004CFD4E
:42A4BE0000000080070000000000000000000000000000000ED00078200000000000000000000000000000000000000000000000000000000000000000000000000000003CFF24
:42A500000000008020010000000000000000000000000000124000080200000000000000000000000000000000000000000000000000000000000000000000000000000068FCB8
:42A54200000000000000000000000000000000000000000000030000040000000000000000000000000000000000000000000000000000000000000000000000000000004CFE86
:42A58400000000800104000000000000000000000000000006C080782000000000000000000000000000000000000000000000000000000000000000000000000000000054FCE2
:42A5C60000000000060200000000000000000000000000000804030100000000000000000000000000000000000000000000000000000000000000000000000000000000E0FC5F
:42A608000000000020000000000000000000000000000000080013001200000000000000000000000000000000000000000000000000000000000000000000000000000094FC33
:42A64A000000008002020000000000000000000000000000024003282000000000000000000000000000000000000000000000000000000000000000000000000000000048FF76
:42A68C00000000000000000000000000000000000000000000000300000000000000000000000000000000000000000000000000000000000000000000000000000000000CFD80
:42A6CE0000000080030000000000000000000000000000001E0403380000000000000000000000000000000000000000000000000000000000000000000000000000000090FEDC
:42A710000800008000010000000000000000000000000000020003081000000000000000000000000000000000000000000000000000000000000000000000000000008004FFDE
:42A7520000000000000000000000000000000000000000004000030004000000000000000000000000000000000000000000000000000000000000000000000000000080C0FD41
:42A7940000000080050400000000000000000000000000001EC883582000000000000000000000000000000000000000000000000000000000000000000000000000000058FCC5
:42A7D600040000000200000000000000000000000000000000000020000000000000000000000000000000000000000000000000000000000000000000000000000000006DFFAF
:42A8180000000000200100000000000000000000000000000004880012000000000000000000000000000000000000000000000000000000000000000000000000000000F4FE4D
:42A85A0000000080020200000000000000000000000000000A4500080000000000000000000000000000000000000000000000000000000000000000000000000000000080FC65
:42A89C00000000000000000000000000000000000000000000000000000000000000000000000000000000000000000000000000000000000000000000000000000000003CFE40
:42A8DE0000000080030000000000000000000000000000000EC003792000000000000000000000000000000000000000000000000000000000000000000000000000000008FC47
:42A92000040000801001000000000000000000000000000042441308020000000000000000000000000000000000000000000000000000000000000000000000000000007DFF41
:42A962000C000000200100000000000000000000000000004000030012000000000000000000000000000000000000000000000000000000000000000000000000000000C8FD6C
:42A9A400000000800500000000000000000000000000000016C880780000000000000000000000000000000000000000000000000000000000000000000000000000000084FF93
:42A9E600080000000200000000000000000000000000000008000000000000000000000000000000000000000000000000000000000000000000000000000000000000809CFC05
:42AA2800000000000001000000000000000000000000000000048B0011000000000000000000000000000000000000000000000000000000000000000000000000000000D4FD7A
:42AA6A00000000800600000000000000000000000000000002400008000000000000000000000000000000000000000000000000000000000000000000000000000000005CFE80
:42AAAC00000000000602000000000000000000000000000000000060000000000000000000000000000000000000000000000000000000000000000000000000000000003CFCC8
:42AAEE0000000000060100000000000000000000000000001EC40361000000000000000000000000000000000000000000000000000000000000000000000000000000005CFE7F
:42AB30000800000026000000000000000000000000000000024110601100000000000000000000000000000000000000000000000000000000000000000000000000008040FD34
:42AB720000000000420200000000000000000000000000008000A0600400000000000000000000000000000000000000000000000000000000000000000000000000008018FC45
:42ABB400000000800700000000000000000000000000000006C4037810000000000000000000000000000000000000000000000000000000000000000000000000000000C4FEC1
:42ABF60004000000060400000000000000000000000000001804006000000000000000000000000000000000000000000000000000000000000000000000000000000000F1FEA4
:42AC380000000000460000000000000000000000000000000000A06012000000000000000000000000000000000000000000000000000000000000000000000000000000FCFF87
:42AC7A000000008000000000000000000000000000000000024000080000000000000000000000000000000000000000000000000000000000000000000000000000000078FC5A
:42ACBC00000000000000000000000000000000000000000000000000000000000000000000000000000000000000000000000000000000000000000000000000000000003CFE1C
:42ACFE00000000000000000000000000000000000000000000C083000000000000000000000000000000000000000000000000000000000000000000000000000000000040FD94
:42AD4000080000000000000000000000000000000000000040442000100000000000000000000000000000000000000000000000000000000000000000000000000000008DFE8A
:42AD82000000000000000000000000000000000000000000400060000400000000000000000000000000000000000000000000000000000000000000000000000000000018FED5
:42ADC400000000800104000000000000000000000000000006C800182000000000000000000000000000000000000000000000000000000000000000000000000000000070FE54
:42AE060004000000060000000000000000000000000000000000030100000000000000000000000000000000000000000000000000000000000000000000000000000080E0FE9E
:42AE480000000000260100000000000000000000000000001804106012000000000000000000000000000000000000000000000000000000000000000000000000000000F4FF10
:42AE8A0000000080000000000000000000000000000000001A41002811000000000000000000000000000000000000000000000000000000000000000000000000000000C0FEB4
:42AECC00000000000000000000000000000000000000000010040000000000000000000000000000000000000000000000000000000000000000000000000000000000006CFFC5
:42AF0E0000000080070200000000000000000000000000001800003820000000000000000000000000000000000000000000000000000000000000000000000000000000A0FF69
:42AF500004000080200000000000000000000000000000001805000802000000000000000000000000000000000000000000000000000000000000000000000000000000A5FE51
:42AF92000C000000C0000000000000000000000000000000580803001200000000000000000000000000000000000000000000000000000000000000000000000000000030FD0F
:42AFD40000000080070000000000000000000000000000001EC0835800000000000000000000000000000000000000000000000000000000000000000000000000000000BCFC43
:42B0160008000000000100000000000000000000000000001800000000000000000000000000000000000000000000000000000000000000000000000000000000000080ACFEAD
:42B058000000000010000000000000000000000000000000580488201100000000000000000000000000000000000000000000000000000000000000000000000000000048FC4D
:42B09A0000000080100000000000000000000000000000001A40030800000000000000000000000000000000000000000000000000000000000000000000000000000000C0FEC1
:42B0DC00000000000001000000000000000000000000000010040300000000000000000000000000000000000000000000000000000000000000000000000000000000005CFDC1
:42B11E00000000000000000000000000000000000000000018D003001000000000000000000000000000000000000000000000000000000000000000000000000000000058FCA0
:42B160000C00000000010000000000000000000000000000184003000100000000000000000000000000000000000000000000000000000000000000000000000000008099FC2F
:42B1A20004000000000000000000000000000000000000001802A00012000000000000000000000000000000000000000000000000000000000000000000000000000080CCFE51
:42B1E40000000080010400000000000000000000000000001EC000180000000000000000000000000000000000000000000000000000000000000000000000000000000068FD49
:42B226000C000000000000000000000000000000000000001804000000000000000000000000000000000000000000000000000000000000000000000000000000000080BDFE83
:42B2680000000000240100000000000000000000000000005800006011000000000000000000000000000000000000000000000000000000000000000000000000000000B0FD09
:42B2AA000000008004000000000000000000000000000000824000081100000000000000000000000000000000000000000000000000000000000000000000000000000064FDA2
:42B2EC000000000006010000000000000000000000000000000400000000000000000000000000000000000000000000000000000000000000000000000000000000000058FDC0
:42B32E00000000000601000000000000000000000000000000000000400000000000000000000000000000000000000000000000000000000000000000000000000000005CFD3D
:42B37000080000001600000000000000000000000000000040040000040000000000000000000000000000000000000000000000000000000000000000000000000000009DFD9B
:42B3B20000000000460000000000000000000000000000004000A00012000000000000000000000000000000000000000000000000000000000000000000000000000000DCFD48
:42B3F400000000800701000000000000000000000000000006C800180000000000000000000000000000000000000000000000000000000000000000000000000000000010FF9A
:42B4360004000000060000000000000000000000000000000000030000000000000000000000000000000000000000000000000000000000000000000000000000000080E0FF68
:42B4780000000000160100000000000000000000000000001004A34011000000000000000000000000000000000000000000000000000000000000000000000000000000DCFE99
:42B4BA00000000000000000000000000000000000000000000000000000000000000000000000000000000000000000000000000000000000000000000000000000000003CFE16
:42B4FC002000048000100002400008000120000480001000024000080001200004000000000010000240000800012000048000100002400008000120000480001000020034FCAC
:42B53E00000000000000000000000000000000000000000000000000000000000000000000000000000000000000000000000000000000000000000000000000000000003CFE91
:42B580002C0004800010000240000800012000048000100002400008000120000400000000001000024000080001200004800010000240000800012000048000100002806DFD61
:42B5C20004000000040000000000000000000000000000001000024000000000000000000000000000000000000000000000000000000000000000000000000000000080C4FDAC
:42B604002000040000100002400008000120000480001000000000000001200004000000000010000240000800012000048000100002400008000120000480001000020070FE2E
:42B646000C00000000000000000000000000000000000000000000000000000000000000000000000000000000000000000000000000000000000000000000000000008065FFD2
:42B688002000048000100002400008000120000480001000024000080001200004000000000010000240000800012000048000100002400008000120000480001000020034FC1E
:42B6CA00000000000000000000000000000000000000000000000000000000000000000000000000000000000000000000000000000000000000000000000000000000003CFE04
:42B70C00000000000000000000000000000000000000000000000000000000000000000000000000000000000000000000000000000000000000000000000000000000003CFEC1
:42B74E0000000000000000000000000000000000000000000800000000000000000000000000000000000000000000000000000000000000000000000000000000000000B4FEFF
:42B79000000000000000000000000000000000000000000000000000000000000000000000000000000000000000000000000000000000000000000000000000000000003CFE3D
:42B7D200000000000000000000000000000000000000000000000000000000000000000000000000000000000000000000000000000000000000000000000000000000003CFEFB
:42B81400000000000000000000000000000000000000000000000000000000000000000000000000000000000000000000000000000000000000000000000000000000003CFEB8
:42B85600000000000000000000000000000000000000000000000000000000000000000000000000000000000000000000000000000000000000000000000000000000003CFE76
:42B89800000000000000000000000000000000000000000000000000000000000000000000000000000000000000000000000000000000000000000000000000000000003CFE34
:42B8DA00000000000000000000000000000000000000000000000000000000000000000000000000000000000000000000000000000000000000000000000000000000003CFEF2
:42B91C00000000000000000000000000000000000000000002000000000000000000000000000000000000000000000000000000000000000000000000000000000000003CFCAF
:42B95E00000000000000000000000000000000000000000000000000000000000000000000000000000000000000000000000000000000000000000000000000000000003CFE6D
:42B9A000000000000000000000000000000000000000000000000000000000000000000000000000000000000000000000000000000000000000000000000000000000003CFE2B
:42B9E200000000000000000000000000000000000000000000000000000000000000000000000000000000000000000000000000000000000000000000000000000000003CFEE9
:42BA2400000000000000000000000000000000000000000000000000000000000000000000000000000000000000000000000000000000000000000000000000000000003CFEA6
:42BA66000000000000000000000000000000000000000000080080000000000000000000000000000000000000000000000000000000000000000000000000000000000034FEE4
:42BAA80000000000020000000000000000000000000000004009012000000000000000000000000000000000000000000000000000000000000000000000000000000000B8FF39
:42BAEA00000000000200000000000000000000000000000000000120000000000000000000000000000000000000000000000000000000000000000000000000000000002CFFCC
:42BB2C00000000000000000000000000000000000000000000000000000000000000000000000000000000000000000000000000000000000000000000000000000000003CFE9D
:42BB6E00000000000000000000000000000000000000000000000000000000000000000000000000000000000000000000000000000000000000000000000000000000003CFE5B
:42BBB000000000000000000000000000000000000000000000000000000000000000000000000000000000000000000000000000000000000000000000000000000000003CFE19
:42BBF200000000000000000000000000000000000000000000000000000000000000000000000000000000000000000000000000000000000000000000000000000000003CFED7
:42BC340000000000800000000000000000000000000000000000000000000000000000000000000000000000000000000000000000000000000000000000000000000000BCFE94
:42BC7600000000000000000000000000000000000000000000000000000000000000000000000000000000000000000000000000000000000000000000000000000000003CFE52
:42BCB800000000000000000000000000000000000000000000000000000000000000000000000000000000000000000000000000000000000000000000000000000000003CFE10
:42BCFA00000000000000000000000000000000000000000000000000000000000000000000000000000000000000000000000000000000000000000000000000000000003CFECE
:42BD3C00000000000000000000000000000000000000000000000000000000000000000000000000000000000000000000000000000000000000000000000000000000003CFE8B
:42BD7E00000000000000000000000000000000000000000000000000000000000000000000000000000000000000000000000000000000000000000000000000000000003CFE49
:42BDC000000000000000000000000000000000000000000000000000000000000000000000000000000000000000000000000000000000000000000000000000000000003CFE07
:42BE0200000000000000000000000000000000000000000000000000000000000000000000000000000000000000000000000000000000000000000000000000000000003CFEC4
:42BE4400000000000000000000000000000000000000000000000000000000000000000000000000000000000000000000000000000000000000000000000000000000003CFE82
:42BE8600000000000000000000000000000000000000000000000000000000000000000000000000000000000000000000000000000000000000000000000000000000003CFE40
:42BEC800000000000000000000000000000000000000000000000000000000000000000000000000000000000000000000000000000000000000000000000000000000003CFEFE
:42BF0A000000000000000000000000000000000000000000024000000000000000000000000000000000000000000000000000000000000000000000000000000000000078FC3F
:42BF4C000000000000000000000000000000000000000000400000000000000000000000000000000000000000000000000000000000000000000000000000000000000038FE3D
:42BF8E00000000000000000000000000000000000000000000000000000000000000000000000000000000000000000000000000000000000000000000000000000000003CFE37
:42BFD000000000000000000000000000000000000000000000000000000000000000000000000000000000000000000000000000000000000000000000000000000000003CFEF5
:42C012000000000000000000000000000000000000000000080081200000000000000000000000000000000000000000000000000000000000000000000000000000000004FD42
:42C05400000000000000000000000000000000000000000000000000000000000000000000000000000000000000000000000000000000000000000000000000000000003CFE70
:42C0960000000000000000000000000000000000000000000480001100000000000000000000000000000000000000000000000000000000000000000000000000000000E0FEF5
:42C0D8000000000000012800000000000000000000000000080001211000000000000000000000000000000000000000000000000000000000000000000000000000000004FEC1
:42C11A000000000000012000000000000000000000000000080001201000000000000000000000000000000000000000000000000000000000000000000000000000000084FF06
:42C15C00000000000000000000000000000000000000000000000000000000000000000000000000000000000000000000000000000000000000000000000000000000003CFE67
:42C19E00000000000000000000000000000000000000000000000000000000000000000000000000000000000000000000000000000000000000000000000000000000003CFE25
:42C1E000000000000000000000000000000000000000000000000000000000000000000000000000000000000000000000000000000000000000000000000000000000003CFEE3
:42C22200000000000000000000000000000000000000000000000000000000000000000000000000000000000000000000000000000000000000000000000000000000003CFEA0
:42C2640000000000010200000000000000000000000000001000000008000000000000000000000000000000000000000000000000000000000000000000000000000000BCFCC5
:42C2A600000000000000000000000000000000000000000000000000000000000000000000000000000000000000000000000000000000000000000000000000000000003CFE1C
:42C2E800000000000000000000000000000000000000000000000000000000000000000000000000000000000000000000000000000000000000000000000000000000003CFEDA
:42C32A00000000000000000000000000000000000000000000000000000000000000000000000000000000000000000000000000000000000000000000000000000000003CFE97
:42C36C00000000000000000000000000000000000000000000000000000000000000000000000000000000000000000000000000000000000000000000000000000000003CFE55
:42C3AE000000008001000000000000000000000000000000008000900000000000000000000000000000000000000000000000000000000000000000000000000000000034FE8A
:42C3F0000000000008000000000000000000000000000000000000000000000000000000000000000000000000000000000000000000000000000000000000000000000034FED1
:42C43200000000000000000000000000000000000000000000000000000000000000000000000000000000000000000000000000000000000000000000000000000000003CFE8E
:42C47400000000000000000000000000000000000000000000000000000000000000000000000000000000000000000000000000000000000000000000000000000000003CFE4C
:42C4B6000004010000000000000000000000000000000000000000000000000000000000000000000000000000000000000000000000000000000000000000000000000038FF08
:42C4F800000100000000000000000000000000000000000000000000000000000000000000000000000000000000000000000000000000000000000000000000000000002CFFD6
:42C53A00000000000000000000000000000000000000000000000000000000000000000000000000000000000000000000000000000000000000000000000000000000003CFE85
:42C57C00000000000000000000000000000000000000000000000000000000000000000000000000000000000000000000000000000000000000000000000000000000003CFE43
:42C5BE000017E002A8000950012A4005A8002DA0025C800B50012A4005A80015400200000000000950012A4005F80115A00254800A50012A800450011240054800092001E8FC60
:42C60000800C9001100106880011200244804010013240068800112002448008800100000000000688001120026482081001224004880011000320020C8008300006C00060FCAA
:02C64200FFFFF8
:00000001FF
